:020000040000FA
:100000000128B501B601B701B801B901A301A501E5
:10001000A401BA01CA01B301B401DB01DC01DE01B4
:10002000DF01CF01BF30DD00640083128501813024
:100030009F00831657309F00303095000F308100AD
:100040000F308500FF23900083122A283008031DFB
:100050003914080089304F2226203918B914B918EC
:10006000B514391085304F22262039183915391921
:100070003515391081304F2226203918B915B91994
:10008000B515391016223E22DC0F4428DD0F442816
:100090000130D000FF30D100FF30D2000130D3005A
:1000A000FF30D400FF30D5000130D600FF30D7003C
:1000B000FF30D800BB28DC0F0800DD0F08005B1CF8
:1000C0005B14BF30DD000800DC0F0800DD0F080006
:1000D0005B185B10BF30DD000800BF0F0800C00FC9
:1000E0000800DB1CDB14CF30C0000800BF0F080085
:1000F000C00F0800DB18DB10CF30C0000800C20FB3
:100100000800C30F08005B1D5B15CF30C30008005B
:10011000BF0F0800C00F08005B195B11CF30C00093
:100120000800C50F0800C60F0800DB1DDB15CF3027
:10013000C6000800BF0F0800C00F0800DB19DB1164
:10014000CF30C0000800DB1C6D20DB187620CF10FC
:10015000DB18CF1408005B1D7F205B1988204F112E
:100160005B194F150800DB1D9120DB199A20CF1178
:10017000DB19CF150800162237183E22DE18A320FF
:100180005E19AB20DE19B3203908031DCD283A10C3
:100190005B1C5B205B186420BB28B91CDD28B814ED
:1001A00089304F22B518FA21CA180A21CA18DA284C
:1001B000B6184C21DF18FE20B810391DED2838156F
:1001C00085304F223519FA214A1920214A19EA2887
:1001D00036194C215F1902213811B91DBB28B815F9
:1001E00081304F22B519FA21CA193621CA19FA28C5
:1001F000B6194C21DF190621B811BB28BE0F080023
:10020000CC210800C10F0800CC210800C40F080051
:10021000CC2108005208031DD20B0800FF30D20089
:100220005108031DD10B0800FF30D100D00B08008E
:10023000FF30D200FF30D1000230D000CA100800D9
:100240005508031DD50B0800FF30D5005408031DC9
:10025000D40B0800FF30D400D30B0800FF30D500CA
:10026000FF30D4000230D3004A1108005808031DA3
:10027000D80B0800FF30D8005708031DD70B080023
:10028000FF30D700D60B0800FF30D800FF30D70072
:100290000230D600CA1108003308AA003008000056
:1002A000AA0200002A08000003185D290000300897
:1002B000B3003108B4006D2108003408AA003108E9
:1002C0000000AA0200002A08000003188C29000080
:1002D00031080000B4006D210800B81874293819DD
:1002E0007C29B81984290800CA142030BE00FF30C8
:1002F000BF00FF30C00008004A152030C100FF30A9
:10030000C200FF30C3000800CA152030C400FF300F
:10031000C500FF30C6000800B81893293819A8296D
:10032000B819BA2908004008031DC00B0800FF30A7
:10033000C0003F08031DBF0B0800FF30BF003E0890
:100340000319A429BE0B0800B610DF14BE01080073
:100350004308031DC30B0800FF30C3004208031D00
:10036000C20B0800FF30C200C10B080036115F1538
:10037000C10108004608031DC60B0800FF30C60077
:100380004508031DC50B0800FF30C500C40B08005D
:10039000B611DF15C40108001130A90030080000B3
:1003A000A9020000290800000318D729EA29B81873
:1003B000DE293819E229B819E6290800DE14B91037
:1003C000DF1008005E1539115F110800DE15B91144
:1003D000DF110800B818F1293819F429B819F729DC
:1003E0000800B910DF10080039115F110800B911B9
:1003F000DF1108000830A90030080000A902000041
:10040000290800000318052A08003A14B8180D2A14
:100410003819102AB819132A0800B510B6140800A4
:10042000351136150800B511B6150800A301B61828
:10043000A315B5182315DF182315CF182315361962
:1004400023163519A3165F19A3164F19A316B6194B
:100450002317B519A317DF19A317CF19A3173A1834
:10046000A3145B1823142308AA002408AA022A084C
:100470000319080037142308A40008002408A50065
:100480000830A1000512A51B051600008516000006
:100490008512A50DA10B422A0512371008009F00F6
:1004A0001530FF3E031D512A9F149F18552A1E0820
:1004B000A70083161E088312A6005F2208002608E4
:1004C000A8002708A9001330AE000310AB01AC014F
:1004D000AD01A80DA90DAD0DAC0DAB0DAE0B762A7F
:1004E00000002C08B0002D08B10008002D30840059
:1004F00080222C30840080222B3084008022692AC4
:1005000003300007AA00AA19800030300007AA00B3
:06051000AA1B800000346C
:02400E00C43FAD
:00000001FF
